:0E00000027C055C0FDCFFCCFFBCFFACF6AC0A2
:10000E00F8CFF7CF4EC0F5CFF4CFF3CFF2CFF1CF7D
:10001E00F0CFEFCFEECFEDCF1027E80364000A004C
:10002E0001000010000110000100010001002D4E22
:10003E00414E0000010002003800010075013A0037
:10004E000000F894EE27ECBBF1E0FBBFEBBFE5BF81
:10005E00F8E1F1BDE1BD8DE0A2E0BB27ED938A95FD
:10006E00E9F780E094E0A0E6ED930197E9F7E2E48A
:10007E00F0E085919591009761F0A591B59105906D
:10008E001590BF01F00105900D920197E1F7FB016C
:10009E00F0CFEFE5EDBFE4E0EEBFC0E6D1E097C1F3
:1000AE0018956A937A93AA93BA93EA93FA93EFB751
:1000BE00EA93A0E6B1E089D4EF5FFF4F6F4F7F4F19
:1000CE008ED4E991EFBFF991E991B991A991799106
:1000DE00699118950A921A92FA926A937A938A9370
:1000EE009A93AA93BA93EA93FA93EFB7EA93EAB57F
:1000FE00FBB5E851FC4FFBBDEABD7394E4E0E71598
:10010E0010F4E1E07E2EF40131964F01EAEFF0E0BB
:10011E008E169F0608F4C6C0E0916001F091610151
:10012E006091620170916301A0E0B1E080E090E027
:10013E00F4D3DF01CB01E2B7EDD1E2D3CBD3E09321
:10014E006901F0936A0160936B0170936C01E0E0BA
:10015E00E2BFE0916901F0916A0160916B017091CB
:10016E006C01C9D3E0936D01F0936E0160936F0142
:10017E0070937001D1D1A130E0E0BE07E0E08E07B0
:10018E00E0E09E0710F0D1D108F008C0D7D1A8EE5C
:10019E00B3E080E090E0DBD1E1E0DFD1C6D110F03A
:1001AE00E0D108F008C0CAD1A4E6B0E080E090E04B
:1001BE00CED1E2E0D2D1D5D110F0DCD108F008C01A
:1001CE00BDD1AAE0B0E080E090E0C1D1E3E0C5D1BE
:1001DE00D1D110F0D8D108F004C0B0D1DDD1E1E01A
:1001EE00E0D1D1D110F0E1D108F009C095D1EAE00B
:1001FE00F0E060E070E0B6D3CFD1E2E0D2D1D5D15D
:10020E0048F08AD1E4E6F0E060E070E0ABD3C4D110
:10021E00E3E0C7D1D3D1E0E0F0E06AE774E4D7D1F0
:10022E00A5E6B1E0D7D1E091650174D1A8EEB3E0B7
:10023E0094D3D3D1E0E0F0E068EC72E4C8D1A6E646
:10024E00B1E0C8D1E0916601A4E6EA02F001C5D1A1
:10025E00E0E0F0E060E271E4BAD1A7E6B1E0BAD135
:10026E00E0916701AAE0EA02F001A8D149D368D271
:10027E00CAD399D2E0937101F09372016093730126
:10028E0070937401BBD336D1A8E6B1E0A3D1E0E000
:10029E00E0936001E0936101E0936201E0936301FA
:1002AE0088249924E991EFBFF991E991B991A99127
:1002BE009991899179916991F99019900990189570
:1002CE009AD19ED1A0D1A7D1AAD1AA98AAD1AD98E0
:1002DE00AB98A998A4D1AA98ABD19DD1909890D162
:1002EE00AA9AADD10895A89AC29AC19A94D197D1DB
:1002FE008AD197D19DD1A3D1C298C198A8980895BB
:10030E00E881E03019F487D18AD1AA98A881A1306A
:10031E0021F471D19198AC98AA98A881A23039F4A1
:10032E00AD9AAB9AA998909A919AAC98AA9AA881EC
:10033E00A33029F470D1909A9198AC98AA9AA8817A
:10034E00A43011F458D184D1A881A53029F4AD9AE6
:10035E00AB98A99A909A7CD1A881A63029F4AD9A2F
:10036E00AB98A99A5CD1AA9AA881A73029F453D147
:10037E0090989198AC98AA98A881A83019F44BD16E
:10038E004ED1AA9AA881A93019F445D1909A60D17C
:10039E001CC0A881A13021F4C09A97989698959880
:1003AE00A881A23021F4C098979A96989598A88122
:1003BE00A33021F4C0989798969A9598A881A43066
:1003CE0021F4C09897989698959A21960895E0E012
:1003DE00E8BBE7E0E7BBE0E0E5BBEFE3E4BBE0E072
:1003EE00E2BBE3EEE1BBE7E0E3BFE0E0E2BFEFBD7F
:1003FE00E2E0EEBDE0E0EDBDECBDE7BDE6BDE9E05F
:10040E00EBBDE4ECEABDE0E0E9BDE8BDE2BDE5BD73
:10041E00E4BDE3BDE5BFE1E1E9BFE0E8E8B9E0E056
:10042E00E0BF789444245524E4E6F0E04E165F06CF
:10043E0028F459DFF20131962F01F6CF44245524CA
:10044E00EAEFF0E04E165F0628F43ADFF20131963D
:10045E002F01F6CFE0EDF7E0FA93EA93FFD0E0E05C
:10046E00E0936401E0936501E0936601E093670118
:10047E00E093680120FE0EC0E72D4CD0EC59FE4FE4
:10048E00E081EA933DDF7A9284DFA898761409F42E
:10049E00A89AF0CFFFCF7B816A81F981E88177FB43
:1004AE00770F67FD7160972F9E5781F078F0983126
:1004BE0090F4AA27BB27882708948795B795A79508
:1004CE009A95D1F7EA23FB23682305C0E894772792
:1004DE00EE27FF2766276F77769508F4606877F921
:1004EE00A991B99189919991EA17FB076807790744
:1004FE0097FB0895B1D082D2CEDF7BD211F4ACD06F
:10050E0007C0EEF7A9D0A0E0B0E080E89FE34BD1A2
:10051E0024960895F0E00895A0916D01B0916E01BA
:10052E0080916F01909170010895F6DFAA30E0E09E
:10053E00BE07E0E08E07E0E09E070895E0916D01B2
:10054E00F0916E0160916F01709170010895E5D187
:10055E00A1E7B1E0F3D03ED208956E2EC29AC198B3
:10056E000895DADFA436E0E0BE07E0E08E07E0E0B3
:10057E009E070895D1DFA83EE3E0BE07E0E08E07B8
:10058E00E0E09E070895C8DFA031E7E2BE07E0E095
:10059E008E07E0E09E070895A1E7B1E0CFD01AD212
:1005AE0008956E2EC298C19A0895B6DFA03AE6E875
:1005BE00BE07E1E08E07E0E09E070895A09171016D
:1005CE00B0917201809173019091740108953DD1A3
:1005DE0015D290CF7CD0EC930895F0DF91D1B0D0AE
:1005EE0012D2E1D0E0937101F09372016093730126
:1005FE0070937401E3CFAD98AB9AA99A9098089531
:10060E00919AAC9A0895AA9A9598C09AE5E0F0E06E
:10061E00FA93EA9323C0AD9AAB9AA99A0895909A49
:10062E00EFCFC098979AE5E0F0E0FA93EA9316C000
:10063E00969A9798E5E0F0E0FA93EA930FC0959AB0
:10064E009698E5E0F0E0FA93EA9308D0959808952D
:10065E009198AC9AAA9A0895C7D10895E991F99103
:10066E00309639F088EE93E00197F1F7A89531971F
:10067E00C9F70895552342F4503811F4E0FF04C031
:10068E003196691F791F6BF050E8572711F45F936D
:10069E00CAC05F3F31F0660F000C57956795752FF6
:1006AE0008955F9300200AF0CAC0C3C050E8192E07
:1006BE001522880F991F9527550F879550E8072EFD
:1006CE000522660F771F7527550F67950895689455
:1006DE0001C0E8945F93F2DF703818F07F3F08F4A2
:1006EE00A2C056E1571BAAF4519558300EF459305A
:1006FE0030F0EFEFFFEF6FEF7FE777F91AC0772754
:10070E005523B9F0EE0FFF1F661F771F5A95D1F7CD
:10071E0010C07727583028F0EF2FF62F672F58503C
:10072E00F9CF552331F076956795F795E7955A955C
:10073E00D1F700200AF4D7D05F910895689401C0D4
:10074E00E894309760407040B1F0002426F0772393
:10075E0012F40094C8D0172E7EE1112032F07A9553
:10076E00EE0FFF1F661F111CF9CFEF2FF62F612D15
:10077E005F938ADF5F9108954F93AF01FD01DA0118
:10078E00AB01BC01CA01402D012C142E4F910895CE
:10079E00EA0FFB1F681F0895E095F0956095EF5FD7
:1007AE00FF4F6F4F08955F9381DF903849F150E806
:1007BE001526703821F1572F591B2BF112F4DCDF5F
:1007CE00FACF583118F0AA27BB278827583028F0BF
:1007DE00AB2FB82F88275850F9CF552329F086957F
:1007EE00B795A7955A95D9F7502D512572F0D0DFB0
:1007FE0038F46795F795E795739513F420C0BCDF31
:10080E0043DF5F910895D8F7FBCFEA1BFB0B680B14
:10081E0051F010F40094C0DF662392F3EE0FFF1F29
:10082E00661F7A95CBF7EE27FF27662777275F910E
:10083E000895EFEFFFEF6FE77FEF5F910895EFEF12
:10084E00FFEF6FE77FE75F9108955F932FDF7038BB
:10085E0021F411200AF4EDCFF2CF903809F4E3CF52
:10086E0001240894970B1BF4D4F30020F3CF792FB7
:10087E001F932F933F934F93112411272227332732
:10088E004427552790E2AE17BF078607410730F081
:10089E00AE1BBF0B860B410B089401C08894551FED
:1008AE00221F331F111CAA1FBB1F881F441F9A959E
:1008BE0051F7F901612D4F913F912F911F916623B1
:1008CE0032F0550FEE1FFF1F661F7A9543F2D2DEF0
:1008DE005F910895EA0FFB1F681F791F0895F19528
:1008EE00E195F0400895F09560957095E195FF4F74
:1008FE006F4F7F4F0895EE0FFF1F661F771F0895EE
:10090E006F2F660F660B762F0895FA9FF02DEB9FD3
:10091E00F00DEA9FE02DF10D08957A9F702D6B9FDB
:10092E00700DF89F700DE99F700D6A9F602D710D0F
:10093E00FB9F600D711DE89F600D711D8827FA9F4A
:10094E00F02D610D781FEB9FF00D611D781FEA9F52
:10095E00E02DF10D681F781F089529D0D6DF0EF413
:10096E00BEDF08953F934F935F93002411244427D5
:10097E00552730E2AA0FBB1F881F991F001C111CA0
:10098E00441F551F0E1A1F0A460B570B28F40E0E46
:10099E001F1E461F571F01C0A1603A9559F7FD0152
:1009AE00BC01D001CA015F914F913F910895E89427
:1009BE00F7FF02C094DF6894B7FF06C0A095B0950C
:1009CE00119600F8039400FA0895ED91FD916D9142
:1009DE007D910895ED93FD936D937C9308957E9391
:1009EE006E93FE93EE930895E881F9816A817B817F
:1009FE000895E883F9836A837B8308957A936A93D3
:100A0E00FA93EA930895182E862F612D192E972F9B
:100A1E00712D1B2EBF2FF12D1A2EAE2FE12D089505
:00000001FF
